:020000040000FA
:020000001228C4
:08000800D000030ED1008312A9
:100010008B1C0B288B1081010B11510E8300D00E0D
:10002000500E09008316FF23900083163F30850091
:10003000383087008312FF308500FE30870083123E
:1000400007309900831600309100831648308100F4
:10005000831231309000831600308C0083121030F0
:100060008B00203084008001840A60300402031C6D
:10007000332881018E018F010B118B100B108C0125
:10008000A0162013A0136400201A8710201E8714C6
:10009000A01A0711A01E0715051C25140518251008
:1000A000251C5728A5140C300F07A4005B28240832
:1000B0000F020319A510A51C2010A518201401304B
:1000C000851CA006051EA014051AA010851E20156B
:1000D000851A2011A011A018A0152019A0150C1C1C
:1000E00073280C10A10AA0198328201B7C28C83073
:1000F0000F07A20020178E2822080F02031D8E284A
:100100002012A0128E282013A01A8E28201A8E28C2
:10011000A01C8C28A0168E2820192016201C96289A
:10012000A013A01A0714A01E07104328A01E071032
:10013000A01E4328A01BA12803302107A300A0175D
:0C0140004328230821020319071043285C
:084000000F000F000F000F007C
:02400E00CC01E3
:00000001FF
